:1000000019C018951895189518951895189518955C
:10001000189518951895706F6465782036384843A0
:1000200031322042444D203C6D7040647563682E2F
:10003000637A3E00F8948FED8DBF8CE087BB8FEF25
:1000400088BB929A8A9A8B9887E089B988E18AB9A5
:1000500083E080936F00552742E16CD181E080936B
:10006000620080E080936100C29AC398F1D1C39A84
:10007000183030F1012F16FD08C017FD03C0FCD168
:1000800032D2F2CFF9D134D2EFCF107E103E21F42C
:10009000D4D1AFD1D7D1E8CF103C39F4CED1D8D11B
:1000A000612FD6D1712FB0D1DFCF103619F4B7D16F
:1000B000C9D1DACF103419F4C0D1B8D1D5CF4EC0E0
:1000C000113091F4C198B99AC098B89A3AE01BD20D
:1000D000B99830916200332309F4339514D2B19B5F
:1000E000FECFC09AB898C0CF123019F4C198B99A0F
:1000F000BBCF133011F4B998B7CF143089F1153054
:10010000D9F4A6D1A12EA4D1B12EA2D1C12EA0D1B5
:10011000D12E08EE6ED1E62EF72E6C21C61639F4DC
:100120007D21D71621F4CE24C094DF24D09414E18D
:10013000E6D010E0E4D098CF163021F489D11093A6
:10014000600092CF173039F483D1A12E81D1B12E26
:1001500014E0D5D089CF103009F486CFC29885CF6E
:1001600077D1103019F417EC83D17ECF113051F4D0
:1001700013E87ED104EE4FEF51E03BD1172F78D139
:10018000A8D072CF1230F9F463D1F12E56D1242FBA
:10019000352F002411242224332400E16DD1A8D16D
:1001A00001E0000E0027101E201E301E03E637D18E
:1001B000C62ED72E839B19C00F2D047029F4D31699
:1001C000C20699F004C028C00316120671F012E0AE
:1001D0000F2D017079F40F2D0870F9F214E048D159
:1001E0001C2D46D11D2D44D1D8CF12E80F2D027001
:1001F00009F01064E12E3CD16CD00E2D007441F05A
:10020000102D36D1112D34D1122D32D1132D30D1E4
:100210000E2D007811F228CF133071F468D058F009
:1002200008EEE7D00FD192E080E0590F481F31501F
:10023000B8F72150A8F718CF143011F509D1109351
:100240006F00143089F05527103011F44EE910C0BA
:10025000113011F44EE40CC0123011F446E208C023
:10026000133011F442E104C04091700050917100CC
:1002700061D0EED010936100EBD010936200F4CE09
:10028000153029F4E5D018BB1FEF17BBEDCE1630A3
:1002900089F42DD070F008ECDBD0612FD9D0712F0C
:1002A000B3D092E080E0590F481F3150A0F72150A1
:1002B00090F7DACE173061F4CBD0BFD04093700006
:1002C0005093710010916F00141509F433D0CCCE07
:1002D00045CF43E6042FA3D0B5D043954836D0F39D
:1002E00004EE4FEF56E085D0162FC2D00895A5D06A
:1002F000AFD0212FADD0312F315020400895612F44
:10030000626011D008EC4A2D5B2D6C2D7D2D7CD0C8
:10031000612F636008D03AE0F6D0612F626003D0AD
:10032000612F01D0089500EC4091600053EF762FCB
:100330006BD00895A42EB52ECC24AA0CBB1CCC1CCB
:10034000AA0CBB1CCC1C002437E0A30EB01CC01CA4
:1003500039E0932EE1D0A02CB12CC22C03E5302E35
:1003600017E0412E20E0522E36E033D060926B0031
:1003700002EE14E036E02DD0639460926A0001E74B
:1003800012E0222734E025D06092690060926C0070
:1003900039E01FD060926D0033E01BD060926E0098
:1003A000300E411E521E00E117E220E036E911D066
:1003B000609263007092640030E40BD0609265003C
:1003C0007092660030E205D060926700709268001B
:1003D0000895932EA1D0001A110A220A632C742CBE
:1003E000852C869477946794060C171C281CA4D03F
:1003F000089542D0042F40D0052F3ED074D042D073
:10040000602F40D0702F089537D0042F35D0052F9E
:1004100033D0062F31D0072F2FD065D008952CD0A0
:100420006CD030D0602F2ED0702F089525D0042F9F
:1004300023D0052F21D061D008950AD0412F08D0B4
:10044000512F0895162F14D0172F12D00895929A75
:100450008399FECF92988399FACF5F9BFCCF1CB112
:10046000929A839BFECF08955F9BFECF1CB10895A7
:100470005D9BFECF1CB9089588E0001F09D08A95C6
:10048000E1F7089588E01BD0001F8A95E1F70895F1
:10049000D0906C00E0906D00F0906E00B89A20F063
:1004A000C098DA94F1F704C0C098DA94F1F7C09AD2
:1004B000EA94F1F7C09AFA94F1F7B8980895D090B9
:1004C0006900E0906A00F0906B008894B89AC09838
:1004D000DA94F1F7B898EA94F1F7B0990894FA949D
:1004E000F1F7C09A0895809163009091640010C064
:1004F00080916500909166000BC08091670090919B
:10050000680006C003D03150E8F7089581EF98E005
:1005100081509040E8F7089500241124222438E007
:10052000990C18F40A0C1B1C2C1C3A9521F0000C99
:10053000111C221CF5CF0895662477248824FF24FB
:10054000F394330C441C551C28F0031414042504A4
:10055000B8F78894579447943794031414042504E7
:1005600020F00318140825086394FA9421F0660C0F
:08057000771C881CEFCF0895F1
:00000001FF
